:0C00000017C0FECFFDCFFCCFFBCFFACF26
:10000C00F9CFF8CFF7CFF6CFF5CFF4CFF3CFF2CFC0
:10001C00F1CFF0CFEFCFEECFEDCF0000010003001A
:10002C0026000000F894EE27ECBBE5BFF8E1A8959C
:10003C00A4B7A77FA4BFF1BDE1BD8DE0A2E0ED9315
:10004C008A95E9F780E8A0E6ED938A95E9F7E8E26E
:10005C00F0E085919591009761F0A591B59105908F
:10006C001590BF01F00105900D920197E1F7FB018E
:10007C00F0CFE0E0E3BBE4BBE5BBEFEDEDBFC0E8E8
:10008C00DCC0E0E0E0BFE3BFE2BFE6BFECBFEFBD2A
:10009C00EEBDEDBDECBDE5BDE4BDEBBDEABDE9BD1E
:1000AC00E8BDEBBFE5BFE9BFEDB9EAB9E0E8E8B9F7
:1000BC00E0E0E1B908956CD100E010E00439E1E131
:1000CC001E0780F4A0E09099A1E0E1E0EA2711F48A
:1000DC00909801C0909A84EF91E00197F1F70F5F2F
:1000EC001F4FECCFA0E09099A1E0E0E0EA2711F4DB
:1000FC00909801C0909A099119910895AA93A8819A
:10010C00A13019F4C79AC69805C0A881A23011F481
:10011C00C798C69AF4D0C798C6982196089536D138
:10012C0020E030E0C39AC49AC19AEDEF3E22D998F0
:10013C00C2DF10E0143008F059C0A1E0E3D0A1E018
:10014C00DDDF969AC59AA12FB0E0E8EEF3E00BD173
:10015C00E053F84F9F01839B02C0220F331FD9013C
:10016C00E4D0C5989698ACEDB5E0DFD0A2E0CAD04B
:10017C00A2E0C4DFA8ECB0E0D8D0849903C0E8E0DA
:10018C003E2A01C0C3D0A0EABFE0CFD033FE20C0CE
:10019C00EFEE3E229298B09B13C02197E0E0E883EB
:1001AC00A881A83760F4849902C0A9D004C0E0E10A
:1001BC003E2AACD004C0E881EF5FE883F1CF2196F2
:1001CC00849905C0E8E03E2AC29AD89A18C00CC09F
:1001DC00E0E13E2A929A6FDF859903C090D0859B0F
:1001EC000EC0A0E4BFE1A1D01F5FA4CF34FE07C0B6
:1001FC00C298D8989698C598C498C198929ACBD022
:10020C00249608957CD085990BC0C298A4EFB1E0D8
:10021C0080D0EFEE3E227AD081D09298C498C198CB
:10022C0008957FD076D072D0EFEE3E2277D0A0E248
:10023C00BEE47BD0C498C1980895E0E8E6BDE0E048
:10024C00E6BDEBBBE3E0EABBE0E0E8BBEEEFE7BB0F
:10025C00C09AE0E0E2BB939AE5ECE1BB12DF2BDF46
:10026C00A4EFB1E062D05AD0C498859906C059D099
:10027C005CD0C398D99A4AD051D0859904C034FE29
:10028C0002C033FE01C002C0BDDF37C0859902C079
:10029C0033FC01C008C0A0EDB7E047D0859902C07F
:1002AC000ADFBFDF2AC0849B04C0859B02C033FCDD
:1002BC0001C00CC024D0849B08C033D036D0D89851
:1002CC00E0E13E2A929A22D02ADF17C0859B04C017
:1002DC0031FE02C033FE01C010C02197E0E0E8837C
:1002EC00A881A43038F40BD0859B04C0E881EF5F63
:1002FC00E883F6CF859913DF2196BFCFFFCFA8EE09
:10030C00B3E013C0FBDEA4EFB1E00FC0E7EF3E2279
:10031C0008950BD0D898C398D99A0895E2E03E2A54
:10032C000895C298ACE2B1E00895109639F080EDD2
:10033C0097E00197F1F7A8951197C9F70895F195F2
:10034C00E195F04008950A2E1B2E81E1AA27BB1BD4
:10035C0005C010F4A00DB11DB695A795F795E795BE
:10036C008A95B9F7089504D0EEDF0EF4E8DF08950E
:10037C00E894F7FF02C0E3DF6894B7FF06C0A095CE
:10038C00B095119600F8039400FA08953A932A93C5
:10039C001A930A9308953B812A8119810881089543
:00000001FF
